:020000040800F2
:1000000090060020150300081D0300081F030008C8
:100010002103000823030008250300080000000056
:10002000000000000000000000000000270300089E
:1000300029030008000000002B0300082D0300081E
:100040002F0300082F0300082F0300082F030008C8
:100050002F0300082F0300082F0300082F030008B8
:100060002F0300082F0300082F0300082F030008A8
:100070002F0300082F0300082F0300082F03000898
:100080002F0300082F0300082F03000800000000C2
:100090000000000000000000000000002F03000826
:1000A0002F0300082F0300082F0300082F03000868
:1000B0002F0300082F0300082F0300082F03000858
:1000C0002F0300082F0300082F0300082F03000848
:1000D0002F0300082F0300082F0300082F03000838
:1000E0002F0300082F0300082F0300080000000062
:1000F0000000000000000000000000000000000000
:1001000000000000000000000000000000000000EF
:1001100000000000000000002F0300082F0300086B
:1001200000F002F800F03AF80AA090E8000C8244CF
:100130008344AAF10107DA4501D100F02FF8AFF2AC
:10014000090EBAE80F0013F0010F18BFFB1A43F0B5
:10015000010318477C5C00009C5C0000103A24BF3F
:1001600078C878C1FAD8520724BF30C830C144BF1C
:1001700004680C607047000000230024002500265E
:10018000103A28BF78C1FBD8520728BF30C148BFFA
:100190000B6070471FB51FBD10B510BD02F01DFDEF
:1001A0001146FFF7F7FF00F085FE02F03BFD03B4B8
:1001B000FFF7F2FF03BC02F043FD00004D4882B0A0
:1001C000016841F00101016041684B4A1140416002
:1001D000016821F4102121F080710160016821F48F
:1001E00080210160416821F4FE0141604FF41F014C
:1001F0008160002201920092016841F48031016027
:10020000016801F4003100910199491C01910099A4
:1002100019B90199B1F5A06FF2D1016811F4003F4D
:1002200008BF009233D00121009134490A6842F09E
:1002300010020A600A6822F003020A600A6842F0AB
:1002400002020A604168416041684160416841F4CE
:1002500080614160416821F47C114160416841F452
:10026000E8114160016841F080710160016811F09E
:10027000007FFBD0416821F003014160416841F0FB
:1002800002014160416801F00C010829FAD11C49C2
:100290004FF00060086002B0704716494868194A7C
:1002A00010F00C03184818BF042B01D0082B01D004
:1002B000026015E04A684B6802F470124FF0020CBD
:1002C00013F4803F0CEB924203D04B6813F4003FD1
:1002D00003D00E4B5A43026002E00A4B5A430260BD
:1002E00049680B4AC1F30311515C026822FA01F11B
:1002F00001607047001002400000FFF8002002403B
:1003000008ED00E000127A000000002000093D0026
:10031000040000200948804709480047FEE7FEE73F
:10032000FEE7FEE7FEE7FEE7FEE7FEE7FEE7FEE7A5
:1003300004480549054A064B70470000BD01000806
:10034000210100089000002090060020900200206B
:100350009002002010B5A0F18041B1F584311DD08C
:10036000B1F5806124D0B1F580612BD0B1F5806109
:1003700032D0B1F5806139D0B1F5806140D0B1F5AE
:10038000806118BF10BD0121080200F066FABDE8C7
:10039000104000214FF4807000F05FBA012104206A
:1003A00000F05BFA0021BDE81040042000F055BACF
:1003B0000121082000F051FA0021BDE8104008207A
:1003C00000F04BBA0121102000F047FA0021BDE8EF
:1003D0001040102000F041BA0121202000F03DFA29
:1003E0000021BDE81040202000F037BA0121402054
:1003F00000F033FA0021BDE81040402000F02DBA93
:100400000121802000F029FA0021BDE81040802061
:1004100000F023BA10B50121084600F01EFA0021B1
:10042000BDE81040012000F018BA2DE9F003CB78A8
:1004300003F00F0213F0100F1CBF8B781A430B78D8
:100440004FF00F0713F0FF0F4FF001081ED00468A4
:10045000002308250E8808FA03FC3CEA060611D1A1
:100460009E0007FA06F924EA090402FA06F6344364
:10047000CE78282E08BFC0F814C003D0482E08BF7D
:10048000C0F810C05B1C6D1EE4D104600B88FF2B0C
:100490009CBFBDE8F003704744684FF0000C08258E
:1004A0000CF108030E8808FA03F333EA060607D0B6
:1004B0006D1E0CF1010CF3D14460BDE8F0037047F0
:1004C0004FEA8C0607FA06F924EA090402FA06F64E
:1004D0003443CE78282E08BF4361CE78482E08BF1B
:1004E0000361E5E74FF6FF7101800221817004216D
:1004F000C17070470246002092680A4218BF01206E
:100500007047806880B2704702460020D2680A4275
:1005100018BF01207047C06880B270470161704702
:1005200041617047002A14BF016141617047C16099
:10053000704741F4803282618161826181698069A2
:1005400070472C4A13684FF6807C03EA0C0343EA99
:1005500000100843106070472749C861704770B4A5
:10056000244A10F0004F14BFD3695368C0F303440A
:100570004FF4401C3CEA00054FEA505C4FEA0C1C6B
:1005800086B206FA0CFC16D010F4801F08BF23EACE
:100590000C0303D0032505FA04F4A34343F070636E
:1005A000002918BF4CEA030310F0004F14BFD361B9
:1005B000536070BC7047546823F0706324F070641B
:1005C0005460EDE78A0721F0030101F1804101F554
:1005D0008031120F0F23D1F808C093402CEA030397
:1005E0008B608B6890401843886070470249C1F85F
:1005F000DC0070470000014000002042AD48016867
:1006000041F0010101604168AB4A1140416001685D
:1006100021F4102121F080710160016821F4802112
:100620000160416821F4FE0141604FF41F018160C7
:100630007047A0490A6822F480320A600A6822F4EE
:1006400080220A60B0F5803F04BF086840F4803023
:1006500006D0B0F5802F06BF086840F4A020704790
:1006600008607047002243099249012B08BF0968BE
:1006700003D0022B0CBF096A496A00F01F00012356
:1006800003FA00F0084218BF01221046704781B0FB
:1006900000208849009000200A6812F4003F18BF2B
:1006A0000120009A521C0092B2F5A06F01D00028E0
:1006B000F1D0086810F4003018BF012001B0704775
:1006C0007C490A6822F0F80242EAC00008607047DC
:1006D0007A4908607047774A5368084323F47C13CB
:1006E00018435060704775490866704771494A68F9
:1006F00022F003021043486070476E48406800F0E3
:100700000C0070476B494A6822F0F00210434860C1
:10071000704768494A6822F4E062104348607047B5
:1007200064494A6822F4605242EAC0004860704757
:10073000604A0029517A14BF084321EA0000507230
:1007400070475E49C1F8D80070475A494A6822F498
:1007500040421043486070475649002281F82020EB
:1007600081F82020012803D004280CBF0520704701
:1007700081F8200070475249086070474D490A6A65
:100780001043086270474F4908607047494910B4E8
:100790004A6812F00C034C4A18BF042B01D0082BF6
:1007A00001D0026015E04A684B6802F470124FF005
:1007B000020C13F4803F0CEB924203D04B6813F40D
:1007C000003F03D0414B5A43026002E03E4B5A4384
:1007D00002604A680F2303EA12123D4B9A5CD0F87C
:1007E00000C02CFA02F24260D1F804C0072404EAE7
:1007F0001C2C13F80CC022FA0CFCC0F808C0D1F86D
:1008000004C004EADC2C13F80C30DA40C2604968FA
:10081000032303EA91312F4B595CB2FBF1F10161E3
:1008200010BC7047234A0029516914BF084321EACC
:100830000000506170471F4A0029916914BF0843A6
:1008400021EA0000906170471A4A0029D16914BF5B
:10085000084321EA0000D0617047164A0029D16898
:1008600014BF084321EA0000D0607047114A0029F4
:10087000116914BF084321EA00001061704716494E
:10088000086070470D49C86470470A49C8717047CD
:100890000848416A41F0807141627047054A01464B
:1008A000002092680A4218BF0120704701498872EF
:1008B00070470000001002400000FFF800004242B4
:1008C000800442423C04424200127A0000093D008A
:1008D00018000020140000204004424210B5A0F18E
:1008E0008041B1F5983111D011F5784119D0B1F5A9
:1008F000806118BF10BD0121C803FFF7B7FFBDE835
:10090000104000214FF40040FFF7B0BF0121080361
:10091000FFF7A3FFBDE8104000214FF48050FFF720
:100920009CBF01218803FFF7A1FFBDE81040002113
:100930004FF48040FFF79ABF10B402880B88B1F8DB
:1009400002C0CC8843EA0C03B1F804C002F441525F
:100950004CEA040C43EA0C03B1F808C043EA0C0368
:10096000B1F80AC043EA0C03B1F80CC043EA0C0327
:10097000B1F80EC043EA0C031A430280828B22F4C2
:1009800000628283098A018210BC7047F0B5054677
:100990000C4602200021AA8B85B0012622F0BF025E
:1009A00022F47062AA832884AF8BA268022A28D01E
:1009B000A088002818BF02266846FFF7E7FEE188F6
:1009C0000098B1F5007F2DD07101B0FBF1F000EB84
:1009D0008000A1684000B0FBF1F0401D80B2684982
:1009E0004FF6FF72A1FB0010C00800F00101401A91
:1009F000C0F34F0002EA0121821EFE2A24BF02201A
:100A00000021E28808431043288420886188A28955
:100A10000843A18811430843384340F40060A88389
:100A200005B0F0BD000A00EB8000A1684000B0FBFB
:100A3000F1F0401D80B2D2E7002101804180818029
:100A4000C180018141818181C1810721018270477B
:100A50000021018041808180C180022282608181E9
:100A600070470029018814BF41F0400121F0400186
:100A7000018070470029818B14BF41F4806121F40B
:100A80008061818370470909012303FA01F1002A7B
:100A9000828889B214BF114322EA01018180704724
:100AA000002A828814BF114322EA01018180704725
:100AB0008181704780897047A1F57E420188FF3AA5
:100AC00014BF41F4807121F48071018070470029C6
:100AD000818814BF41F0040121F004018180704736
:100AE000028822F40062028002881143018070476C
:100AF000018841F48051018070470029018814BFAA
:100B000041F4005121F4005101807047012914BFC4
:100B1000008B808A7047008A7047B1F5804F01884A
:100B20000CBF41F4804121F48041018070470246AE
:100B3000002012890A4218BF01207047C943018171
:100B4000704701F00F034FF0010C0CFA03F3002281
:100B500009090CFA01F1B0F804C09BB289B200890E
:100B60000CEA010118421CBF0029012210467047FF
:100B700001F00F01012202FA01F1C943018170471E
:100B8000CDCCCCCCA0F1804110B5B1F5A8414FF04F
:100B9000010109D08805FFF769FEBDE8104000217A
:100BA0004FF48000FFF762BE4FF40010FFF75EFEC7
:100BB000BDE8104000214FF40010FFF757BE70B59C
:100BC0000446808886B00D4620F03F066846FFF751
:100BD000DDFDB2490298B0FBF1F189B246EA0102AB
:100BE000A280228822F001022280AD4B2A689A421C
:100BF0001DD85200B0FBF2F080B2042838BF0420A8
:100C0000491C2184A083208840F001002080208896
:100C1000A9886A8920F00A0020F480601143084303
:100C20002080A88929890843208106B070BDEB88FF
:100C3000A3F53F4CBCF1FF0C19D002EBC20303EB50
:100C40000212B0FBF2F080B240F480400205120DB7
:100C500008BF40F0010040F400404FF49672514349
:100C60004FF47A72B1FBF2F1491C2184CAE702EB1E
:100C70004202B0FBF2F080B2E8E741F28831016055
:100C8000002181804BF6FF72C280018141814FF4C7
:100C90008041818170470029018814BF41F0010122
:100CA00021F00101018070470029818814BF41F4BF
:100CB000006121F40061818070470029818814BFA0
:100CC00041F4805121F480518180704700290188CE
:100CD00014BF41F4807121F48071018070470029B4
:100CE000018814BF41F4007121F400710180704744
:100CF0000029018814BF41F4806121F480610180E2
:100D00007047828901F0FE0122F0FE0211438181C9
:100D100070470029818914BF41F0010121F00101D0
:100D2000818170470029018814BF41F0400121F002
:100D3000400101807047002A828814BF114322EAD3
:100D400001018180704701827047008AC0B27047FC
:100D5000002A14BF41F0010101F0FE010182704739
:100D600081B008440090008801B0704700290188D4
:100D700014BF41F40041C1F30E0101807047B1F589
:100D8000006F01880CBF41F4006121F40061018013
:100D90007047B1F5005F01880CBF41F4005121F4A8
:100DA0000051018070470029018814BF41F480512F
:100DB00021F4805101807047B1F5006F01880CBFAC
:100DC00041F4006121F4006101807047002901882D
:100DD00014BF41F0200121F0200101807047008BF9
:100DE000000A70470029018814BF41F0100121F06A
:100DF000100101807047002901880CBF41F080017B
:100E000021F0800101807047B1F5804F818B14BFC4
:100E100021F4804141F4804181837047838A00221C
:100E2000008B43EA004020F07F4031EA000008BF19
:100E3000012210467047818A008B41EA004020F071
:100E40007F40704782B00246002000920A0F21F0D6
:100E50007F41019208BF090C009A14BF1432183266
:100E6000009212680A4218BF012002B07047C943BD
:100E700081827047838800224FF4E06C0CEA114CA9
:100E8000808A03EA0C0321F07F4108421CBF002B3B
:100E9000012210467047C9438182704740420F00CB
:100EA000A0860100002100EBC000884288BF491CD9
:100EB000FBD8704782B000F07FF800F0B8F800F07F
:100EC00013FE00F0E5F80025F0234FF4A072294648
:100ED0002846009500F06EF9012000F004F9032186
:100EE000002001F0CBFD4FF6FF73CC22002127A09C
:100EF000009500F0D5FD1F21202001F0BFFD33211A
:100F0000212001F0BBFD274C0E2001F0F6FD2070E2
:100F10000F2001F0F2FD607010F0800F4FF6FF73AC
:100F20004FF0E0024FF00001009514BF1EA020A07A
:100F300000F0B6FD2078002200F00F0020706178EC
:100F40004FF4FC6301F03F01617000EB01101146AA
:100F500000F0E3FB4CF25031002001EBC101814273
:100F600088BF401CFBD80C2001F0C7FD20700D206D
:100F700001F0C3FD607021784FF6E07301EB0020B3
:100F80006422002100F0C9FBBEE70000415033326B
:100F9000313620414C532C50532B49522D4C454453
:100FA00000000000280000204F626A6563740000A2
:100FB000202020202020000070B501210420FFF710
:100FC0003AFC01210820FFF736FC01210846FFF713
:100FD00032FC01215748FFF7C2FA01215648FFF7BA
:100FE000BEFA564CA020564D20800320A070182039
:100FF000E07021462846FFF718FA402020800420A0
:10100000E07021462846FFF710FA40F202402080A7
:101010000220A0701020E07021464A4C2046FFF7C5
:1010200004FA21152046BDE87040FFF777BA10B5E5
:10103000012186B00803FFF7FEFB0020ADF8000099
:10104000ADF808004FF48271ADF80400ADF80C0063
:10105000ADF80210ADF80600ADF80E004FF40071C7
:101060000720394CADF80A10ADF81000694620464B
:10107000FFF762FCA1152046FFF71EFD0021204668
:10108000FFF73BFD01212046FFF7EBFC06B010BD4A
:1010900010B5012184B04805FFF7D6FB01210846B1
:1010A000FFF7C9FB2548022181701C21C170C021B6
:1010B000018001462348FFF7B8F96846FFF7DDFDD8
:1010C000224800900120ADF808008002204CADF8C5
:1010D0000A0069462046FFF772FD01212046FFF70E
:1010E000DAFD04B010BD10B514490122154C0A8078
:1010F00080B1012816D0022818BF10BD1020C8707A
:101100000E492046FFF791F92046BDE81040012125
:10111000FFF704BA2820C8702046BDE810400749F0
:10112000FFF783B94820C8702046BDE81040034946
:10113000FFF77BB900013000000230002A000020D8
:1011400000080140000C014000300140A086010071
:101150000054004070B505460221FE48FFF7DEF955
:10116000FD4C02212046FFF7E2FC0028F9D0294679
:101170002046FFF79DFC80212046FFF7D8FC012880
:10118000F9D070BD70B505460221F248FFF7C8F9E5
:10119000F14C02212046FFF7CAFC0028F9D029466D
:1011A0002046FFF785FC80212046FFF7C0FC012880
:1011B000F9D070BD2DE9F05FE64D0F460646984622
:1011C00092464FF0360B02212846DDF82890FFF7B3
:1011D000A7F9E14C02212046FFF7A9FC0028F9D02D
:1011E00059462046FFF764FC80212046FFF79FFC0C
:1011F0000128F9D04FF0E80B02212846FFF78EF9BD
:1012000002212046FFF793FC0028F9D059462046DA
:10121000FFF74EFC80212046FFF789FC0128F9D01A
:101220004FF02A0B02212846FFF77AF902212046C7
:10123000FFF77DFC0028F9D059462046FFF738FC1F
:1012400080212046FFF773FC0128F9D04FEA162BC6
:1012500002212846FFF762F902212046FFF767FCCA
:101260000028F9D059462046FFF722FC802120466D
:10127000FFF75DFC0128F9D006F0FF0B022128469C
:10128000FFF74CF902212046FFF751FC0028F9D066
:1012900059462046FFF70CFC80212046FFF747FC0B
:1012A0000128F9D006EB0A00461EC6F3072B0221DF
:1012B0002846FFF733F902212046FFF738FC0028C3
:1012C000F9D059462046FFF7F3FB80212046FFF76F
:1012D0002EFC0128F9D0F6B202212846FFF71EF9AC
:1012E00002212046FFF723FC0028F9D03146204692
:1012F000FFF7DEFB80212046FFF719FC0128F9D01B
:101300002B2602212846FFF70BF902212046FFF782
:101310000EFC0028F9D031462046FFF7C9FB80219A
:101320002046FFF704FC0128F9D0002602212846B8
:10133000FFF7F4F802212046FFF7F9FB0028F9D067
:1013400031462046FFF7B4FB80212046FFF7EFFB34
:101350000128F9D002212846FFF7E0F802212046B3
:10136000FFF7E5FB0028F9D039462046FFF7A0FB40
:1013700080212046FFF7DBFB0128F9D0002602215F
:101380002846FFF7CBF802212046FFF7D0FB0028C4
:10139000F9D031462046FFF78BFB80212046FFF72E
:1013A000C6FB0128F9D007EB0800401EC6B2022197
:1013B0002846FFF7B3F802212046FFF7B8FB0028C4
:1013C000F9D031462046FFF773FB80212046FFF716
:1013D000AEFB0128F9D02C2602212846FFF7A0F801
:1013E00002212046FFF7A3FB0028F9D03146204612
:1013F000FFF75EFB80212046FFF799FB0128F9D01B
:1014000002212846FFF78AF800250AFB08F6002E7D
:101410008CBF4FEA1927BDE8F09F02212046FFF755
:1014200086FB0028F9D039462046FFF741FB022110
:101430002046FFF77CFB0028F9D049462046FFF7FD
:1014400037FB6D1CAE42E8D8BDE8F09F2DE9F84FA0
:10145000404E88460546994617464FF0360A022107
:101460003046DDF828B0FFF75BF83B4C0221204600
:10147000FFF75DFB0028F9D051462046FFF718FB27
:1014800080212046FFF753FB0128F9D04FF0E80AEE
:1014900002213046FFF742F802212046FFF747FBC2
:1014A0000028F9D051462046FFF702FB8021204654
:1014B000FFF73DFB0128F9D04FF02A0A0221304600
:1014C000FFF72EF802212046FFF731FB0028F9D064
:1014D00051462046FFF7ECFA80212046FFF727FB14
:1014E0000128F9D0C8F3072A02213046FFF716F881
:1014F00002212046FFF71BFB0028F9D05146204669
:10150000FFF7D6FA80212046FFF711FB0128F9D01A
:1015100008F0FF0A02213046FFF700F802212046BA
:10152000FFF705FB0028F9D051462046FFF7C0FA27
:1015300080212046FFF7FBFA0128F9D008F13F0887
:10154000C8F3072A02213046FEF7E8FF02212046B1
:1015500004E00000000C014000300140FFF7E7FA12
:101560000028F3D051462046FFF7A2FA80212046FA
:10157000FFF7DDFA0128F9D008F0FF080221304614
:10158000FEF7CCFF02212046FFF7D1FA0028F9D060
:1015900041462046FFF78CFA80212046FFF7C7FA24
:1015A0000128F9D04FF02B0802213046FEF7B8FF92
:1015B00002212046FFF7BBFA0028F9D04146204619
:1015C000FFF776FA80212046FFF7B1FA0128F9D01B
:1015D0004FF0000802213046FEF7A0FF022120460E
:1015E000FFF7A5FA0028F9D041462046FFF760FA38
:1015F00080212046FFF79BFA0128F9D007F0FF0869
:1016000002213046FEF78AFF02212046FFF78FFABB
:101610000028F9D041462046FFF74AFA80212046AB
:10162000FFF785FA0128F9D04FF000080221304673
:10163000FEF774FF02212046FFF779FA0028F9D05F
:1016400041462046FFF734FA80212046FFF76FFA23
:101650000128F9D007F16300C7B202213046FEF736
:101660005DFF02212046FFF762FA0028F9D03946D3
:101670002046FFF71DFA80212046FFF758FA01287F
:10168000F9D02C2702213046FEF74AFF02212046DE
:10169000FFF74DFA0028F9D039462046FFF708FA3F
:1016A00080212046FFF743FA0128F9D00221304675
:1016B000FEF734FF05EBC50000EB0510DFF88CA446
:1016C000002700900098002507EB40181FFA8BF6C2
:1016D0001AF80800A84010F0800F18BF1FFA89F60A
:1016E00080212046FFF723FA0128F9D0310A20464D
:1016F000FFF7DEF980212046FFF719FA0128F9D01B
:1017000031462046FFF7D4F96D1C082DDED37F1C2F
:10171000B7F5487FD6D3BDE8F88F2DE9FF4F0D46CA
:1017200042F21071B0FBF1F111F0FF066FF41C7181
:1017300006FB01F100EB01104FF47A71B0FBF1F1FF
:1017400001F0FF096FF07C0109FB01F100EBC10022
:10175000FF4981B0A1FB0021C1F347186FF01801C8
:1017600008FB01F100EB8100FA494FF00004A1FBF6
:101770000021C1F3C707C7F1000101EB810100EBB4
:101780004100039A9B4600F0FF0A009429460CBFD3
:101790000B203046FFF75AFE039A56EA09065B46CD
:1017A000009405F140010CBF0B204846FFF74EFEA8
:1017B000039A56EA08065B46009405F180010CBFC7
:1017C0000B204046FFF742FE039A56EA07005B46AD
:1017D000009405F1C0010CBF0B203846FFF736FE20
:1017E0005B46009405F580715046039AFFF72EFE84
:1017F00005B0BDE8F08F2DE9FF5FD74F0E46984644
:1018000015464FF0360902213846DDF838A0FEF7BC
:1018100087FED24C02212046FFF789F90028F9D033
:1018200049462046FFF744F980212046FFF77FF91B
:101830000128F9D04FF0E80902213846FEF76EFE84
:1018400002212046FFF773F90028F9D049462046C7
:10185000FFF72EF980212046FFF769F90128F9D01A
:101860004FF02A0902213846FEF75AFE022120468F
:10187000FFF75DF90028F9D049462046FFF718F92F
:1018800080212046FFF753F90128F9D04FEA1629A5
:1018900002213846FEF742FE02212046FFF747F9B3
:1018A0000028F9D049462046FFF702F9802120465A
:1018B000FFF73DF90128F9D006F0FF09022138466B
:1018C000FEF72CFE02212046FFF731F90028F9D05F
:1018D00049462046FFF7ECF880212046FFF727F91C
:1018E0000128F9D00F36C6F3072902213846FEF742
:1018F00015FE02212046FFF71AF90028F9D04946C3
:101900002046FFF7D5F880212046FFF710F901287F
:10191000F9D0F6B202213846FEF700FE0221204639
:10192000FFF705F90028F9D031462046FFF7C0F847
:1019300080212046FFF7FBF80128F9D02B26022151
:101940003846FEF7EDFD02212046FFF7F0F80028AB
:10195000F9D031462046FFF7ABF880212046FFF74B
:10196000E6F80128F9D0002602213846FEF7D6FD18
:1019700002212046FFF7DBF80028F9D03146204647
:10198000FFF796F880212046FFF7D1F80128F9D01B
:10199000EEB202213846FEF7C1FD02212046FFF7D4
:1019A000C6F80028F9D031462046FFF781F880219B
:1019B0002046FFF7BCF80128F9D00026022138465E
:1019C000FEF7ACFD02212046FFF7B1F80028F9D060
:1019D00031462046FFF76CF880212046FFF7A7F834
:1019E0000128F9D005F10F00C5B202213846FEF7F3
:1019F00095FD02212046FFF79AF80028F9D02946E4
:101A00002046FFF755F880212046FFF790F801287F
:101A1000F9D02C2502213846FEF782FD022120460E
:101A2000FFF785F80028F9D029462046FFF740F84F
:101A300080212046FFF77BF80128F9D002213846A3
:101A4000FEF76CFDDFF818B100270098002607EBC1
:101A5000401955461BF80900B04010F0800F18BF20
:101A6000454680212046FFF762F80128F9D0290A6F
:101A70002046FFF71DF880212046FFF758F801287F
:101A8000F9D029462046FFF713F8701C86B2082EBD
:101A9000DFD3781C87B2202FD7D304B0BDE8F09FE6
:101AA0002DE9F84F064600250078DDF82880994694
:101AB00092460F462C46002808BFBDE8F88F7819DB
:101AC00081B2CDF80080305D4B462038C0B252461E
:101AD000FFF791FE05F1100085B2601C84B2305D05
:101AE0000028ECD1BDE8F88F70B51B4D4FF4806134
:101AF0002846FEF715FD42F21070FFF7D3F92915BD
:101B00002846FEF70BFD012602212846FEF708FDB8
:101B1000124C02212046FFF70AF80028F9D031467E
:101B20002046FEF7C5FF80212046FFF700F8012878
:101B3000F9D042F21070FFF7B5F9CB260221284602
:101B4000FEF7EEFC022120460CE000004E380008B3
:101B50001F85EB51CDCCCCCC000C014000300140B6
:101B60004E2C0008FEF7E3FF0028EBD0314620465C
:101B7000FEF79EFF80212046FEF7D9FF0128F9D00D
:101B8000392602212846FEF7C9FC02212046FEF72D
:101B9000CEFF0028F9D031462046FEF789FF80218C
:101BA0002046FEF7C4FF0128F9D02C260221284642
:101BB000FEF7B4FC02212046FEF7B9FF0028F9D059
:101BC00031462046FEF774FF80212046FEF7AFFF26
:101BD0000128F9D0002602212846FEF79FFC0221A9
:101BE0002046FEF7A4FF0028F9D031462046FEF734
:101BF0005FFF80212046FEF79AFF0128F9D03426A6
:101C000002212846FEF78AFC02212046FEF78FFFBC
:101C10000028F9D031462046FEF74AFF80212046B1
:101C2000FEF785FF0128F9D0022631462846FEF747
:101C300075FC02212046FEF77AFF0028F9D03146D4
:101C40002046FEF735FF80212046FEF770FF012871
:101C5000F9D0CF2602212846FEF762FC0221204659
:101C6000FEF765FF0028F9D031462046FEF720FF39
:101C700080212046FEF75BFF0128F9D000260221D3
:101C80002846FEF74BFC02212046FEF750FF0028B5
:101C9000F9D031462046FEF70BFF80212046FEF7A3
:101CA00046FF0128F9D0C12602212846FEF736FC5E
:101CB00002212046FEF73BFF0028F9D0314620469E
:101CC000FEF7F6FE80212046FEF731FF0128F9D00D
:101CD000302602212846FEF721FC02212046FEF78D
:101CE00026FF0028F9D031462046FEF7E1FE80218C
:101CF0002046FEF71CFF0128F9D0E82602212846DD
:101D0000FEF70EFC02212046FEF711FF0028F9D055
:101D100031462046FEF7CCFE80212046FEF707FF25
:101D20000128F9D0852602212846FEF7F7FB02217B
:101D30002046FEF7FCFE0028F9D031462046FEF78B
:101D4000B7FE80212046FEF7F2FE0128F9D00026DA
:101D500002212846FEF7E2FB02212046FEF7E7FEBD
:101D60000028F9D031462046FEF7A2FE8021204609
:101D7000FEF7DDFE0128F9D0782602212846FEF77D
:101D8000CDFB02212046FEF7D2FE0028F9D03146D5
:101D90002046FEF78DFE80212046FEF7C8FE012872
:101DA000F9D0EA2602212846FEF7BAFB0221204696
:101DB000FEF7BDFE0028F9D031462046FEF778FE3A
:101DC00080212046FEF7B3FE0128F9D0002602212B
:101DD0002846FEF7A3FB02212046FEF7A8FE0028B6
:101DE000F9D031462046FEF763FE80212046FEF7FB
:101DF0009EFE0128F9D0002602212846FEF78EFB20
:101E000002212046FEF793FE0028F9D031462046F5
:101E1000FEF74EFE80212046FEF789FE0128F9D00C
:101E2000ED2602212846FEF77BFB02212046FEF725
:101E30007EFE0028F9D031462046FEF739FE80218B
:101E40002046FEF774FE0128F9D0642602212846B8
:101E5000FEF764FB02212046FEF769FE0028F9D058
:101E600031462046FEF724FE80212046FEF75FFE25
:101E70000128F9D0032602212846FEF74FFB022154
:101E80002046FEF754FE0028F9D031462046FEF7E2
:101E90000FFE80212046FEF74AFE0128F9D01226C7
:101EA00002212846FEF73AFB02212046FEF73FFEBC
:101EB0000028F9D031462046FEF7FAFD8021204661
:101EC000FEF735FE0128F9D0812602212846FEF7CB
:101ED00025FB02212046FEF72AFE0028F9D03146D4
:101EE0002046FEF7E5FD80212046FEF720FE012872
:101EF000F9D0F72602212846FEF712FB02212046E0
:101F0000FEF715FE0028F9D031462046FEF7D0FD39
:101F100080212046FEF70BFE0128F9D02026022161
:101F20002846FEF7FBFA02212046FEF700FE0028B5
:101F3000F9D031462046FEF7BBFD80212046FEF752
:101F4000F6FD0128F9D0C02602212846FEF7E8FA5E
:101F500002212046FEF7EBFD0028F9D0314620464D
:101F6000FEF7A6FD80212046FEF7E1FD0128F9D00D
:101F7000232602212846FEF7D1FA02212046FEF749
:101F8000D6FD0028F9D031462046FEF791FD80218C
:101F90002046FEF7CCFD0128F9D0C12602212846B3
:101FA000FEF7BEFA02212046FEF7C1FD0028F9D057
:101FB00031462046FEF77CFD80212046FEF7B7FD26
:101FC0000128F9D0102602212846FEF7A7FA02219F
:101FD0002046FEF7ACFD0028F9D031462046FEF73A
:101FE00067FD80212046FEF7A2FD0128F9D0C52615
:101FF00002212846FEF794FA02212046FEF797FDBB
:102000000028F9D031462046FEF752FD80212046B7
:10201000FEF78DFD0128F9D03E2602212846FEF765
:102020007DFA02212046FEF782FD0028F9D03146D4
:102030002046FEF73DFD80212046FEF778FD012871
:10204000F9D0282602212846FEF768FA0221204608
:10205000FEF76DFD0028F9D031462046FEF728FD39
:1020600080212046FEF763FD0128F9D0C726022112
:102070002846FEF755FA02212046FEF758FD0028B3
:10208000F9D031462046FEF713FD80212046FEF7A9
:102090004EFD0128F9D0862602212846FEF73EFA99
:1020A00002212046FEF743FD0028F9D031462046A4
:1020B000FEF7FEFC80212046FEF739FD0128F9D00D
:1020C000362602212846FEF72BFA02212046FEF78B
:1020D0002EFD0028F9D031462046FEF7E9FC80218C
:1020E0002046FEF724FD0128F9D0E82602212846E3
:1020F000FEF714FA02212046FEF719FD0028F9D058
:1021000031462046FEF7D4FC80212046FEF70FFD25
:102110000128F9D03A2602212846FEF701FA0221C9
:102120002046FEF704FD0028F9D031462046FEF790
:10213000BFFC80212046FEF7FAFC0128F9D0552685
:1021400002212846FEF7EAF902212046FEF7EFFCBD
:102150000028F9D031462046FEF7AAFC802120460F
:10216000FEF7E5FC0128F9D0B12602212846FEF74A
:10217000D7F902212046FEF7DAFC0028F9D03146D3
:102180002046FEF795FC80212046FEF7D0FC012872
:10219000F9D0002602212846FEF7C0F90221204688
:1021A000FEF7C5FC0028F9D031462046FEF780FC3A
:1021B00080212046FEF7BBFC0128F9D01826022119
:1021C0002846FEF7ABF902212046FEF7B0FC0028B6
:1021D000F9D031462046FEF76BFC80212046FEF701
:1021E000A6FC0128F9D0B62602212846FEF798F968
:1021F00002212046FEF79BFC0028F9D031462046FC
:10220000FEF756FC80212046FEF791FC0128F9D00C
:10221000082602212846FEF781F902212046FEF712
:1022200086FC0028F9D031462046FEF741FC80218B
:102230002046FEF77CFC0128F9D0822602212846A0
:10224000FEF76CF902212046FEF771FC0028F9D058
:1022500031462046FEF72CFC80212046FEF767FC25
:102260000128F9D0272602212846FEF757F9022136
:102270002046FEF75CFC0028F9D031462046FEF7E8
:1022800017FC80212046FEF752FC0128F9D0F226E7
:1022900002212846FEF744F902212046FEF747FCBA
:1022A0000028F9D031462046FEF702FC8021204666
:1022B000FEF73DFC0128F9D0002602212846FEF752
:1022C0002DF902212046FEF732FC0028F9D03146D4
:1022D0002046FEF7EDFB80212046FEF728FC012872
:1022E000F9D02A2602212846FEF71AF902212046B3
:1022F000FEF71DFC0028F9D031462046FEF7D8FB3A
:1023000080212046FEF713FC0128F9D00026022187
:102310002846FEF703F902212046FEF708FC0028B4
:10232000F9D031462046FEF7C3FB80212046FEF758
:10233000FEFB0128F9D0002602212846FEF7EEF820
:1023400002212046FEF7F3FB0028F9D03146204653
:10235000FEF7AEFB80212046FEF7E9FB0128F9D00D
:10236000012602212846FEF7D9F802212046FEF771
:10237000DEFB0028F9D031462046FEF799FB80218C
:102380002046FEF7D4FB0128F9D03F26022128463B
:10239000FEF7C4F802212046FEF7C9FB0028F9D059
:1023A00031462046FEF784FB80212046FEF7BFFB26
:1023B0000128F9D02B2602212846FEF7B1F8022188
:1023C0002046FEF7B4FB0028F9D031462046FEF740
:1023D0006FFB80212046FEF7AAFB0128F9D00026DA
:1023E00002212846FEF79AF802212046FEF79FFBBD
:1023F0000028F9D031462046FEF75AFB80212046BE
:10240000FEF795FB0128F9D0002602212846FEF7A9
:1024100085F802212046FEF78AFB0028F9D03146D4
:102420002046FEF745FB80212046FEF780FB012871
:10243000F9D0002602212846FEF770F80221204636
:10244000FEF775FB0028F9D031462046FEF730FB39
:1024500080212046FEF76BFB0128F9D0EF260221F0
:102460002846FEF75BF802212046FEF760FB0028B5
:10247000F9D031462046FEF71BFB80212046FEF7AF
:1024800056FB0128F9D0262602212846FEF748F8F7
:1024900002212046FEF74BFB0028F9D031462046AA
:1024A000FEF706FB80212046FEF741FB0128F9D00C
:1024B000012602212846FEF731F802212046FEF7C8
:1024C00036FB0028F9D031462046FEF7F1FA80218C
:1024D0002046FEF72CFB0128F9D0E02602212846F1
:1024E000FEF71EF802212046FEF721FB0028F9D056
:1024F00031462046FEF7DCFA80212046FEF717FB26
:102500000128F9D00F2602212846FEF707F80221FC
:102510002046FEF70CFB0028F9D031462046FEF796
:10252000C7FA80212046FEF702FB0128F9D03126A8
:1025300002212846FDF7F2FF02212046FEF7F7FAB6
:102540000028F9D031462046FEF7B2FA8021204615
:10255000FEF7EDFA0128F9D02B2602212846FDF7D7
:10256000DDFF02212046FEF7E2FA0028F9D03146CD
:102570002046FEF79DFA80212046FEF7D8FA012872
:10258000F9D00C2602212846FDF7C8FF022120467B
:10259000FEF7CDFA0028F9D031462046FEF788FA3A
:1025A00080212046FEF7C3FA0128F9D00E26022129
:1025B0002846FDF7B3FF02212046FEF7B8FA0028AF
:1025C000F9D031462046FEF773FA80212046FEF707
:1025D000AEFA0128F9D0082602212846FDF79EFF11
:1025E00002212046FEF7A3FA0028F9D03146204602
:1025F000FEF75EFA80212046FEF799FA0128F9D00D
:102600004E2602212846FDF789FF02212046FEF7CB
:102610008EFA0028F9D031462046FEF749FA80218B
:102620002046FEF784FA0128F9D0F1260221284637
:10263000FDF774FF02212046FEF779FA0028F9D051
:1026400031462046FEF734FA80212046FEF76FFA25
:102650000128F9D0372602212846FDF75FFF022125
:102660002046FEF764FA0028F9D031462046FEF7EE
:102670001FFA80212046FEF75AFA0128F9D00726D2
:1026800002212846FDF74AFF02212046FEF74FFAB5
:102690000028F9D031462046FEF70AFA802120466C
:1026A000FEF745FA0128F9D0102602212846FDF749
:1026B00035FF02212046FEF73AFA0028F9D03146CC
:1026C0002046FEF7F5F980212046FEF730FA012872
:1026D000F9D0032602212846FDF720FF02212046DB
:1026E000FEF725FA0028F9D031462046FEF7E0F93A
:1026F00080212046FEF71BFA0128F9D00E26022180
:102700002846FDF70BFF02212046FEF710FA0028AD
:10271000F9D031462046FEF7CBF980212046FEF75E
:1027200006FA0128F9D0092602212846FDF7F6FE0F
:1027300002212046FEF7FBF90028F9D03146204659
:10274000FEF7B6F980212046FEF7F1F90128F9D00D
:10275000002602212846FDF7E1FE02212046FEF771
:10276000E6F90028F9D031462046FEF7A1F980218C
:102770002046FEF7DCF90128F9D0E126022128469F
:10278000FDF7CEFE02212046FEF7D1F90028F9D050
:1027900031462046FEF78CF980212046FEF7C7F926
:1027A0000128F9D0002602212846FDF7B7FE0221B4
:1027B0002046FEF7BCF90028F9D031462046FEF746
:1027C00077F980212046FEF7B2F90128F9D00E26CC
:1027D00002212846FDF7A2FE02212046FEF7A7F9B6
:1027E0000028F9D031462046FEF762F980212046C4
:1027F000FEF79DF90128F9D0142602212846FDF79D
:102800008DFE02212046FEF792F90028F9D03146CC
:102810002046FEF74DF980212046FEF788F9012871
:10282000F9D0032602212846FDF778FE0221204632
:10283000FEF77DF90028F9D031462046FEF738F939
:1028400080212046FEF773F90128F9D011260221D4
:102850002846FDF763FE02212046FEF768F90028AE
:10286000F9D031462046FEF723F980212046FEF7B5
:102870005EF90128F9D0072602212846FDF74EFE11
:1028800002212046FEF753F90028F9D031462046B0
:10289000FEF70EF980212046FEF749F90128F9D00C
:1028A000312602212846FDF739FE02212046FEF797
:1028B0003EF90028F9D031462046FEF7F9F880218C
:1028C0002046FEF734F90128F9D0C1260221284616
:1028D000FDF724FE02212046FEF729F90028F9D051
:1028E00031462046FEF7E4F880212046FEF71FF926
:1028F0000128F9D0482602212846FDF70FFE0221C3
:102900002046FEF714F90028F9D031462046FEF79C
:10291000CFF880212046FEF70AF90128F9D00826D1
:1029200002212846FDF7FAFD02212046FEF7FFF8B6
:102930000028F9D031462046FEF7BAF8802120461B
:10294000FEF7F5F80128F9D00F2602212846FDF7F9
:10295000E5FD02212046FEF7EAF80028F9D03146CD
:102960002046FEF7A5F880212046FEF7E0F8012872
:10297000F9D00C2602212846FDF7D0FD0221204681
:10298000FEF7D5F80028F9D031462046FEF790F83A
:1029900080212046FEF7CBF80128F9D0312602210C
:1029A0002846FDF7BBFD02212046FEF7C0F80028AF
:1029B000F9D031462046FEF77BF880212046FEF70D
:1029C000B6F80128F9D0362602212846FDF7A6FDE3
:1029D00002212046FEF7ABF80028F9D03146204608
:1029E000FEF766F880212046FEF7A1F80128F9D00D
:1029F0000F2602212846FDF791FD02212046FEF711
:102A000096F80028F9D031462046FEF751F880218B
:102A10002046FEF78CF80128F9D01126022128461D
:102A2000FDF77EFD02212046FEF781F80028F9D04F
:102A300031462046FEF73CF880212046FEF777F825
:102A40000128F9D00C48FEF72DFA29260221284644
:102A5000FDF766FD02212046FEF769F80028F9D04F
:102A600031462046FEF724F880212046FEF75FF825
:102A70000128F9D070BD0000A08601002DE9F041C9
:102A80004F4D0E46044601212846FEF71FF94D4FD3
:102A900028463946FEF7C2F90028F9D000223C2129
:102AA0002846FEF755F9484F28463946FEF7B6F94D
:102AB0000028F9D021462846FEF745F9434C284620
:102AC0002146FEF7ABF90028F9D031462846FEF73B
:102AD0003AF921462846FEF7A1F90028F9D001214C
:102AE0002846FEF7FCF800BF4FF400312846FEF7F9
:102AF000A9F90028F8D1BDE8F0812DE9F041304D69
:102B0000064600BF4FF400312846FEF79BF9002827
:102B1000F8D101212846FEF7D9F82A4C284621464B
:102B2000FEF77CF90028F9D000223C212846FEF768
:102B30000FF9254F28463946FEF770F90028F9D0DD
:102B400031462846FEF7FFF8204E28463146FEF76C
:102B500065F90028F9D001212846FEF7B7F821468B
:102B60002846FEF75BF90028F9D001223C212846CF
:102B7000FEF7EEF8164C28462146FEF74FF90028DE
:102B8000F9D02846FEF7E1F8264607462C4631469E
:102B90002046FEF743F90028F9D000212046FEF731
:102BA000A7F801212046FEF79AF800BF4FF4003144
:102BB0002046FEF747F90028F8D13846BDE8F081F5
:102BC0000054004001000300820007008400070059
:102BD00040000300704770477047754600F02CF8BE
:102BE000AE4605006946534620F00700854618B0FA
:102BF00020B5FDF79DFBBDE820404FF000064FF0EB
:102C000000074FF000084FF0000B21F00701AC4621
:102C1000ACE8C009ACE8C009ACE8C009ACE8C00940
:102C20008D46704710B50446AFF300802046BDE8DE
:102C30001040FDF7BCBA000000487047300000208B
:102C400001491820ABBEFEE72600020070470000D5
:102C50000000000000000000000000000000000074
:102C60000000000000000000000000000000000064
:102C7000000007000F800F800F800F800F8007007B
:102C80000700000000000700070007000000000028
:102C90000E380E380E380E380630000000000000E6
:102CA0000000000000000000000000000000000024
:102CB0000C300C300C307FFE7FFE0C300C300C30B2
:102CC0000C307FFE7FFE0C300C300C30000000001A
:102CD000024002400FF81FF81A401A401FF00FF888
:102CE000025802581FF81FF0024002400000000086
:102CF000000000000E100E300E7000E001C00380D6
:102D000007000E700C70087000000000000000004A
:102D100000000F001980198019800F000F080F980C
:102D200019F818F018E019F00F98000000000000E2
:102D300000000700070007000E0000000000000070
:102D40000000000000000000000000000000000083
:102D5000000000F001C0038007000E000E000E000E
:102D60000E000700038001C000F00000000000001A
:102D700000000F00038001C000E0007000700070D0
:102D8000007000E001C003800F00000000000000A0
:102D9000000001801188099007E007E03FFC3FFC3C
:102DA00007E007E0099011880180000000000000A2
:102DB0000000000000000180018001800FF00FF092
:102DC0000180018001800000000000000000000080
:102DD00000000000000000000000000000000000F3
:102DE000000000000700070007000E0000000000C0
:102DF0000000000000000000000000001FF81FF8A5
:102E000000000000000000000000000000000000C2
:102E100000000000000000000000000000000000B2
:102E20000000000070007000700000000000000052
:102E3000000000020006000E001C0038007000E0D8
:102E400001C0038007000E001C000000000000000D
:102E500000000FF01C381C381C381C381C381C387B
:102E60001C381C381C381C380FF000000000000013
:102E700000000180018003801F801F800380038089
:102E800003800380038003801FF000000000000027
:102E900000000FE01C701C380038007000E001C01A
:102EA000038007000E381C381FF8000000000000E7
:102EB00000000FE01C701C380038007003C003C015
:102EC000007000381C381C700FE00000000000008B
:102ED000000000E001E003E006E00CE018E01FF86D
:102EE0001FF800E000E000E003F800000000000030
:102EF00000001FF81C001C001C001C001FE01FF03D
:102F0000007800381C381C700FE000000000000042
:102F1000000003E007000E001C001C001FF01FF85B
:102F20001C381C381C381C380FF000000000000052
:102F300000001FFC1C1C1C1C1C1C001C003800700A
:102F400000E001C003800380038000000000000057
:102F500000000FF01C381C381C381F3807E007E051
:102F60001CF81C381C381C380FF000000000000052
:102F700000000FF01C381C381C381C381FF80FF8E4
:102F800000380038007000E007C0000000000000BA
:102F900000000000000003800380038000000000A8
:102FA0000380038003800000000000000000000098
:102FB0000000000000000380038003800000000088
:102FC0000380038003800700000000000000000071
:102FD000007000E001C0038007000E001C001C0010
:102FE0000E000700038001C000E000700000000038
:102FF00000000000000000003FFC3FFC000000005B
:103000003FFC3FFC0000000000000000000000004A
:103010001C000E000700038001C000E0007000707B
:1030200000E001C0038007000E001C00000000004B
:1030300003C00FF01E7818380038007000E001C09F
:1030400001C00000000001C001C001C0000000007C
:103050000FF81C1C1C1C1C1C1C1C1CFC1CFC1CFC41
:103060001CFC1C001C001C001FF007F800000000E6
:10307000000003C007E00E701C381C381C381C38D8
:103080001FF81C381C381C381C38000000000000D9
:1030900000001FF00E380E380E380E380FF00FF00B
:1030A0000E380E380E380E381FF0000000000000F9
:1030B000000007F00E381C381C001C001C001C000F
:1030C0001C001C001C380E3807F000000000000037
:1030D00000001FE00E700E380E380E380E380E3815
:1030E0000E380E380E380E701FE000000000000091
:1030F00000001FF80E180E080E000E300FF00FF033
:103100000E300E000E080E181FF800000000000020
:1031100000001FF80E180E080E000E300FF00FF012
:103120000E300E000E000E001F0000000000000018
:10313000000007F00E381C381C381C001C001C0056
:103140001CF81C381C380E3807F80000000000007E
:1031500000001C701C701C701C701C701FF01FF095
:103160001C701C701C701C701C70000000000000A3
:1031700000000FE00380038003800380038003804E
:1031800003800380038003800FE000000000000044
:10319000000001FC00700070007000700070007092
:1031A00038703870387038700FE000000000000090
:1031B00000001E380E380E700EE00FC00F800F801A
:1031C0000FC00EE00E700E381E3800000000000028
:1031D00000001F000E000E000E000E000E000E007C
:1031E0000E000E080E180E381FF800000000000038
:1031F00000001C1C1E3C1F7C1FFC1FFC1DDC1C9CBB
:103200001C1C1C1C1C1C1C1C1C1C000000000000A6
:1032100000001C1C1C1C1E1C1F1C1F9C1DDC1CFCFD
:103220001C7C1C3C1C1C1C1C1C1C00000000000006
:10323000000003E007F00E381C1C1C1C1C1C1C1C8E
:103240001C1C1C1C0E3807F003E0000000000000EE
:1032500000001FF00E380E380E380E380FF00FF049
:103260000E000E000E000E001F0000000000000007
:10327000000003E00F780E381C1C1C1C1C1C1C1CBE
:103280001C7C1CFC0FF80FF8003800FC000000004C
:1032900000001FF00E380E380E380E380FF00FF009
:1032A0000E700E380E380E381E3800000000000078
:1032B00000000FF01C381C381C381C000FE007F011
:1032C00000381C381C381C380FF0000000000000CB
:1032D00000001FFC19CC11C401C001C001C001C015
:1032E00001C001C001C001C007F0000000000000E3
:1032F00000001C701C701C701C701C701C701C70FA
:103300001C701C701C701C700FE00000000000009E
:1033100000001C701C701C701C701C701C701C70D9
:103320001C701C700EE007C003800000000000004D
:1033300000001C1C1C1C1C1C1C1C1C1C1C9C1C9C05
:103340001C9C0FF80FF807700770000000000000C9
:1033500000001C701C701C700EE007C0038003800E
:1033600007C00EE01C701C701C7000000000000004
:1033700000001C701C701C701C701C700EE007C0DC
:1033800003800380038003800FE000000000000042
:1033900000001FF81C381838107000E001C00380CE
:1033A00007000E081C181C381FF800000000000061
:1033B000000007F0070007000700070007000700EC
:1033C000070007000700070007F0000000000000EA
:1033D0000000100018001C000E000700038001C050
:1033E00000E000700038001C000700000000000032
:1033F000000007F000700070007000700070007036
:10340000007000700070007007F000000000000005
:1034100000000000000000001C701C701C701C707C
:103420001C701C701C701FD81C001C001C000000AD
:10343000000000000000000000000000000000008C
:10344000000000000000000000007FFF7FFF000080
:1034500000001C001C000700070000000000000026
:10346000000000000000000000000000000000005C
:10347000000000000000000000000FE0007000707D
:103480000FF01C701C701C700FD8000000000000B2
:1034900000001E000E000E000E000FF00E380E3859
:1034A0000E380E380E380E381BF0000000000000F9
:1034B000000000000000000000000FE01C701C7005
:1034C0001C001C001C701C700FE0000000000000BD
:1034D000000000F80070007000700FF01C701C708D
:1034E0001C701C701C701C700FD8000000000000C5
:1034F000000000000000000000000FE01C701C70C5
:103500001FF01C001C701C700FE000000000000089
:10351000000003E007700770070007001FE01FE0CE
:1035200007000700070007001FC0000000000000A0
:10353000000000000000000000000FD81C701C708C
:103540001C701C700FF007F000701C700FE0000082
:1035500000001E000E000E000E000EF00F380F3897
:103560000E380E380E380E381E38000000000000ED
:10357000000001C001C001C000000FC001C001C0B7
:1035800001C001C001C001C00FF800000000000030
:103590000000007000700070000003F00070007008
:1035A00000700070007000701C700CF007E00000EC
:1035B00000001E000E000E000E000E380E700EE011
:1035C0000FC00EE00E700E381E3800000000000024
:1035D00000000FC001C001C001C001C001C001C096
:1035E00001C001C001C001C00FF8000000000000D0
:1035F000000000000000000000001FF81C9C1C9C44
:103600001C9C1C9C1C9C1C9C1C9C00000000000022
:10361000000000000000000000001FE01C701C7093
:103620001C701C701C701C701C70000000000000DE
:10363000000000000000000000000FE01C701C7083
:103640001C701C701C701C700FE00000000000005B
:10365000000000000000000000001BF00E380E38D3
:103660000E380E380E380FF00E000E001F0000004E
:10367000000000000000000000001FB038E038E04B
:1036800038E038E038E01FE000E000E001F0000042
:10369000000000000000000000001EF00FF80F38CE
:1036A0000E000E000E000E001F00000000000000C3
:1036B000000000000000000000000FE01C301C3083
:1036C0000F8003E0187018700FE000000000000089
:1036D000000000000100030007001FF007000700C2
:1036E000070007000770077003E0000000000000FB
:1036F000000000000000000000001C701C701C7026
:103700001C701C701C701C700FD8000000000000A2
:10371000000000000000000000001C701C701C7005
:103720001C701C700EE007C0038000000000000049
:10373000000000000000000000001C1C1C1C1C1CE1
:103740001C9C1C9C0FF80770077000000000000014
:10375000000000000000000000001CE01CE00FC0A2
:10376000078007800FC01CE01CE000000000000084
:10377000000000000000000000000E380E380E3877
:103780000E380E3807F003E000E001C01F80000093
:10379000000000000000000000001FE018E011C061
:1037A000038007000E201C601FE0000000000000E6
:1037B000000001F803800380038007001C001C0048
:1037C000070003800380038001F800000000000070
:1037D00001C001C001C001C001C001C001C001C0E1
:1037E00001C001C001C001C001C001C00000000053
:1037F00000001F8001C001C001C000E00038003897
:1038000000E001C001C001C01F80000000000000F6
:10381000000000000000000000001F1C3B9C39DC81
:1038200038F8000000000000000000000000000068
:10383000000000F001F80198019801F800F0000084
:103840000000000000000000000000000000000078
:103850000000000000000000000000000000000068
:103860000000000000000000000000000000000058
:103870007FFFFFF800000000FFFFFFFC00000001D9
:10388000FFFFFFFE00000003FFFFFFFF0000000737
:10389000FFFFFFFF80000007FFFFFFFFC0000007E2
:1038A000FFFFFFFF88000023FFFFFFFF1C000071E8
:1038B000FFFFFFFE3E0000F8FFFFFFFC7F0001FC62
:1038C0007FFFFFF8FF8003FE00000001FFC007FF3D
:1038D00000000001FFC007FF00000001FFC007FF5C
:1038E00000000001FFC007FF00000001FFC007FF4C
:1038F00000000001FFC007FF00000001FFC007FF3C
:1039000000000001FFC007FF00000001FFC007FF2B
:1039100000000001FFC007FF00000001FFC007FF1B
:1039200000000001FFC007FF00000001FFC007FF0B
:1039300000000001FFC007FF00000001FFC007FFFB
:1039400000000001FFC007FF00000001FFC007FFEB
:1039500000000001FFC007FF00000001FFC007FFDB
:1039600000000001FFC007FF00000001FFC007FFCB
:1039700000000001FFC007FF00000001FFC007FFBB
:1039800000000001FFC007FF00000001FFC007FFAB
:1039900000000001FFC007FF00000001FFC007FF9B
:1039A000000000007FC007FC000000003FC007F0DF
:1039B000000000000FC007E00000000003C0078007
:1039C0000000000001C006000000000000400000F0
:1039D00000000000000000000000000000000000E7
:1039E00000000000000004000000000000000700CC
:1039F0000000000000C007C00000000003C007F086
:103A0000000000000FC007FC000000003FC007FFDF
:103A100000000000FFC007FF00000001FFC007FF1B
:103A200000000001FFC007FF00000001FFC007FF0A
:103A300000000001FFC007FF00000001FFC007FFFA
:103A400000000001FFC007FF00000001FFC007FFEA
:103A500000000001FFC007FF00000001FFC007FFDA
:103A600000000001FFC007FF00000001FFC007FFCA
:103A700000000001FFC007FF00000001FFC007FFBA
:103A800000000001FFC007FF00000001FFC007FFAA
:103A900000000001FFC007FF00000001FFC007FF9A
:103AA00000000001FFC007FF00000001FFC007FF8A
:103AB00000000001FFC007FF00000001FFC007FF7A
:103AC00000000001FFC007FF00000001FFC007FF6A
:103AD00000000001FFC007FF00000001FFC007FF5A
:103AE00000000001FFC007FF00000001FFC003FE4F
:103AF00000000000FF8001FC000000007F0000F8D3
:103B00007FFFFFF83E000070FFFFFFFC1C0000215C
:103B1000FFFFFFFE08000003FFFFFFFF000000079C
:103B2000FFFFFFFF80000007FFFFFFFFC00000074F
:103B3000FFFFFFFF80000003FFFFFFFF0000000109
:103B4000FFFFFFFE00000000FFFFFFFC0000000081
:103B50007FFFFFF8000000000000000000000000F0
:103B60000000000000000000000000000000000055
:103B70000000000000000000000000000000000045
:103B80000000000000000000000000000000000035
:103B90000000000000000000000000000000000025
:103BA0000000000000000000000000000000000015
:103BB0000000000000000000000000000000000005
:103BC0000000000008000000000000001C000000D1
:103BD000000000003E000000000000007F00000028
:103BE00000000000FF80000000000001FFC0000096
:103BF00000000001FFC0000000000001FFC0000045
:103C000000000001FFC0000000000001FFC0000034
:103C100000000001FFC0000000000001FFC0000024
:103C200000000001FFC0000000000001FFC0000014
:103C300000000001FFC0000000000001FFC0000004
:103C400000000001FFC0000000000001FFC00000F4
:103C500000000001FFC0000000000001FFC00000E4
:103C600000000001FFC0000000000001FFC00000D4
:103C700000000001FFC0000000000001FFC00000C4
:103C800000000001FFC0000000000001FFC00000B4
:103C900000000001FFC0000000000001FFC00000A4
:103CA00000000001FFC0000000000001FFC0000094
:103CB00000000001FFC0000000000001FFC0000084
:103CC000000000007FC00000000000003FC00000B6
:103CD000000000000FC000000000000003C0000052
:103CE0000000000001C000000000000000400000D3
:103CF00000000000000000000000000000000000C4
:103D000000000000000000000000000000000000B3
:103D10000000000000C000000000000003C0000020
:103D2000000000000FC00000000000003FC00000C5
:103D300000000000FFC0000000000001FFC0000004
:103D400000000001FFC0000000000001FFC00000F3
:103D500000000001FFC0000000000001FFC00000E3
:103D600000000001FFC0000000000001FFC00000D3
:103D700000000001FFC0000000000001FFC00000C3
:103D800000000001FFC0000000000001FFC00000B3
:103D900000000001FFC0000000000001FFC00000A3
:103DA00000000001FFC0000000000001FFC0000093
:103DB00000000001FFC0000000000001FFC0000083
:103DC00000000001FFC0000000000001FFC0000073
:103DD00000000001FFC0000000000001FFC0000063
:103DE00000000001FFC0000000000001FFC0000053
:103DF00000000001FFC0000000000001FFC0000043
:103E000000000001FFC0000000000001FFC0000032
:103E100000000000FF800000000000007F000000A4
:103E2000000000003E000000000000001C00000038
:103E3000000000000800000000000000000000007A
:103E40000000000000000000000000000000000072
:103E50000000000000000000000000000000000062
:103E60000000000000000000000000000000000052
:103E70000000000000000000000000000000000042
:103E80000000000000000000000000000000000032
:103E90000000000000000000000000000000000022
:103EA0000000000000000000000000000000000012
:103EB0007FFFFFF800000000FFFFFFFC0000000193
:103EC000FFFFFFFE00000003FFFFFFFF00000007F1
:103ED000FFFFFFFF80000007FFFFFFFFC00000079C
:103EE000FFFFFFFF88000003FFFFFFFF1C00000132
:103EF000FFFFFFFE3E000000FFFFFFFC7F00000011
:103F00007FFFFFF8FF80000000000001FFC00000FD
:103F100000000001FFC0000000000001FFC0000021
:103F200000000001FFC0000000000001FFC0000011
:103F300000000001FFC0000000000001FFC0000001
:103F400000000001FFC0000000000001FFC00000F1
:103F500000000001FFC0000000000001FFC00000E1
:103F600000000001FFC0000000000001FFC00000D1
:103F700000000001FFC0000000000001FFC00000C1
:103F800000000001FFC0000000000001FFC00000B1
:103F900000000001FFC0000000000001FFC00000A1
:103FA00000000001FFC0000000000001FFC0000091
:103FB00000000001FFC0000000000001FFC0000081
:103FC00000000001FFC0000000000001FFC0000071
:103FD00000000001FFC0000000000001FFC0000061
:103FE000000000007FC00000000000003FC0000093
:103FF0007FFFFFFC0FC00001FFFFFFFE03C00007B3
:10400000FFFFFFFF81C0000FFFFFFFFFE040003F09
:10401000FFFFFFFFF80000FFFFFFFFFFFE00007F34
:10402000FFFFFFFFFC00041FFFFFFFFFF00007077B
:10403000FFFFFFFFC00007C1FFFFFFFF000007F009
:104040007FFFFFFC000007FC00000000000007FFEE
:1040500000000000000007FF00000000000007FF54
:1040600000000000000007FF00000000000007FF44
:1040700000000000000007FF00000000000007FF34
:1040800000000000000007FF00000000000007FF24
:1040900000000000000007FF00000000000007FF14
:1040A00000000000000007FF00000000000007FF04
:1040B00000000000000007FF00000000000007FFF4
:1040C00000000000000007FF00000000000007FFE4
:1040D00000000000000007FF00000000000007FFD4
:1040E00000000000000007FF00000000000007FFC4
:1040F00000000000000007FF00000000000007FFB4
:1041000000000000000007FF00000000000007FFA3
:1041100000000000000007FF00000000000007FF93
:1041200000000000000007FF00000000000003FE88
:1041300000000000000001FC00000000000000F88A
:104140007FFFFFF800000070FFFFFFFC0000002170
:10415000FFFFFFFE00000003FFFFFFFF000000075E
:10416000FFFFFFFF80000007FFFFFFFFC000000709
:10417000FFFFFFFF80000003FFFFFFFF00000001C3
:10418000FFFFFFFE00000000FFFFFFFC000000003B
:104190007FFFFFF8000000000000000000000000AA
:1041A000000000000000000000000000000000000F
:1041B00000000000000000000000000000000000FF
:1041C00000000000000000000000000000000000EF
:1041D0007FFFFFF800000000FFFFFFFC0000000170
:1041E000FFFFFFFE00000003FFFFFFFF00000007CE
:1041F000FFFFFFFF80000007FFFFFFFFC000000779
:10420000FFFFFFFF88000003FFFFFFFF1C0000010E
:10421000FFFFFFFE3E000000FFFFFFFC7F000000ED
:104220007FFFFFF8FF80000000000001FFC00000DA
:1042300000000001FFC0000000000001FFC00000FE
:1042400000000001FFC0000000000001FFC00000EE
:1042500000000001FFC0000000000001FFC00000DE
:1042600000000001FFC0000000000001FFC00000CE
:1042700000000001FFC0000000000001FFC00000BE
:1042800000000001FFC0000000000001FFC00000AE
:1042900000000001FFC0000000000001FFC000009E
:1042A00000000001FFC0000000000001FFC000008E
:1042B00000000001FFC0000000000001FFC000007E
:1042C00000000001FFC0000000000001FFC000006E
:1042D00000000001FFC0000000000001FFC000005E
:1042E00000000001FFC0000000000001FFC000004E
:1042F00000000001FFC0000000000001FFC000003E
:10430000000000007FC00000000000003FC000006F
:104310007FFFFFFC0FC00001FFFFFFFE03C000078F
:10432000FFFFFFFF81C0000FFFFFFFFFE040003FE6
:10433000FFFFFFFFF80000FFFFFFFFFFFE00007F11
:10434000FFFFFFFFFC00001FFFFFFFFFF000000763
:10435000FFFFFFFFC0C00001FFFFFFFF03C0000021
:104360007FFFFFFC0FC00000000000003FC0000006
:1043700000000000FFC0000000000001FFC00000BE
:1043800000000001FFC0000000000001FFC00000AD
:1043900000000001FFC0000000000001FFC000009D
:1043A00000000001FFC0000000000001FFC000008D
:1043B00000000001FFC0000000000001FFC000007D
:1043C00000000001FFC0000000000001FFC000006D
:1043D00000000001FFC0000000000001FFC000005D
:1043E00000000001FFC0000000000001FFC000004D
:1043F00000000001FFC0000000000001FFC000003D
:1044000000000001FFC0000000000001FFC000002C
:1044100000000001FFC0000000000001FFC000001C
:1044200000000001FFC0000000000001FFC000000C
:1044300000000001FFC0000000000001FFC00000FC
:1044400000000001FFC0000000000001FFC00000EC
:1044500000000000FF800000000000007F0000005E
:104460007FFFFFF83E000000FFFFFFFC1C00000183
:10447000FFFFFFFE08000003FFFFFFFF0000000733
:10448000FFFFFFFF80000007FFFFFFFFC0000007E6
:10449000FFFFFFFF80000003FFFFFFFF00000001A0
:1044A000FFFFFFFE00000000FFFFFFFC0000000018
:1044B0007FFFFFF800000000000000000000000087
:1044C00000000000000000000000000000000000EC
:1044D00000000000000000000000000000000000DC
:1044E00000000000000000000000000000000000CC
:1044F00000000000000000000000000000000000BC
:1045000000000000000000000000000000000000AB
:10451000000000000000000000000000000000009B
:104520000000000008000020000000001C000070D7
:10453000000000003E0000F8000000007F0001FCC9
:1045400000000000FF8003FE00000001FFC007FF25
:1045500000000001FFC007FF00000001FFC007FFCF
:1045600000000001FFC007FF00000001FFC007FFBF
:1045700000000001FFC007FF00000001FFC007FFAF
:1045800000000001FFC007FF00000001FFC007FF9F
:1045900000000001FFC007FF00000001FFC007FF8F
:1045A00000000001FFC007FF00000001FFC007FF7F
:1045B00000000001FFC007FF00000001FFC007FF6F
:1045C00000000001FFC007FF00000001FFC007FF5F
:1045D00000000001FFC007FF00000001FFC007FF4F
:1045E00000000001FFC007FF00000001FFC007FF3F
:1045F00000000001FFC007FF00000001FFC007FF2F
:1046000000000001FFC007FF00000001FFC007FF1E
:1046100000000001FFC007FF00000001FFC007FF0E
:10462000000000007FC007FC000000003FC007F052
:104630007FFFFFFC0FC007E1FFFFFFFE03C00787FE
:10464000FFFFFFFF81C0060FFFFFFFFFE040003FBD
:10465000FFFFFFFFF80000FFFFFFFFFFFE00007FEE
:10466000FFFFFFFFFC00001FFFFFFFFFF000000740
:10467000FFFFFFFFC0C00001FFFFFFFF03C00000FE
:104680007FFFFFFC0FC00000000000003FC00000E3
:1046900000000000FFC0000000000001FFC000009B
:1046A00000000001FFC0000000000001FFC000008A
:1046B00000000001FFC0000000000001FFC000007A
:1046C00000000001FFC0000000000001FFC000006A
:1046D00000000001FFC0000000000001FFC000005A
:1046E00000000001FFC0000000000001FFC000004A
:1046F00000000001FFC0000000000001FFC000003A
:1047000000000001FFC0000000000001FFC0000029
:1047100000000001FFC0000000000001FFC0000019
:1047200000000001FFC0000000000001FFC0000009
:1047300000000001FFC0000000000001FFC00000F9
:1047400000000001FFC0000000000001FFC00000E9
:1047500000000001FFC0000000000001FFC00000D9
:1047600000000001FFC0000000000001FFC00000C9
:1047700000000000FF800000000000007F0000003B
:10478000000000003E000000000000001C000000CF
:104790000000000008000000000000000000000011
:1047A0000000000000000000000000000000000009
:1047B00000000000000000000000000000000000F9
:1047C00000000000000000000000000000000000E9
:1047D00000000000000000000000000000000000D9
:1047E00000000000000000000000000000000000C9
:1047F00000000000000000000000000000000000B9
:1048000000000000000000000000000000000000A8
:104810007FFFFFF800000000FFFFFFFC0000000129
:10482000FFFFFFFE00000003FFFFFFFF0000000787
:10483000FFFFFFFF80000007FFFFFFFFC000000732
:10484000FFFFFFFF80000023FFFFFFFF000000715C
:10485000FFFFFFFE000000F8FFFFFFFC000001FC6F
:104860007FFFFFF8000003FE00000000000007FFCC
:1048700000000000000007FF00000000000007FF2C
:1048800000000000000007FF00000000000007FF1C
:1048900000000000000007FF00000000000007FF0C
:1048A00000000000000007FF00000000000007FFFC
:1048B00000000000000007FF00000000000007FFEC
:1048C00000000000000007FF00000000000007FFDC
:1048D00000000000000007FF00000000000007FFCC
:1048E00000000000000007FF00000000000007FFBC
:1048F00000000000000007FF00000000000007FFAC
:1049000000000000000007FF00000000000007FF9B
:1049100000000000000007FF00000000000007FF8B
:1049200000000000000007FF00000000000007FF7B
:1049300000000000000007FF00000000000007FF6B
:1049400000000000000007FC00000000000007F06D
:104950007FFFFFFC000007E1FFFFFFFE000007876D
:10496000FFFFFFFF8000060FFFFFFFFFE000003F9B
:10497000FFFFFFFFF80000FFFFFFFFFFFE00007FCB
:10498000FFFFFFFFFC00001FFFFFFFFFF00000071D
:10499000FFFFFFFFC0C00001FFFFFFFF03C00000DB
:1049A0007FFFFFFC0FC00000000000003FC00000C0
:1049B00000000000FFC0000000000001FFC0000078
:1049C00000000001FFC0000000000001FFC0000067
:1049D00000000001FFC0000000000001FFC0000057
:1049E00000000001FFC0000000000001FFC0000047
:1049F00000000001FFC0000000000001FFC0000037
:104A000000000001FFC0000000000001FFC0000026
:104A100000000001FFC0000000000001FFC0000016
:104A200000000001FFC0000000000001FFC0000006
:104A300000000001FFC0000000000001FFC00000F6
:104A400000000001FFC0000000000001FFC00000E6
:104A500000000001FFC0000000000001FFC00000D6
:104A600000000001FFC0000000000001FFC00000C6
:104A700000000001FFC0000000000001FFC00000B6
:104A800000000001FFC0000000000001FFC00000A6
:104A900000000000FF800000000000007F00000018
:104AA0007FFFFFF83E000000FFFFFFFC1C0000013D
:104AB000FFFFFFFE08000003FFFFFFFF00000007ED
:104AC000FFFFFFFF80000007FFFFFFFFC0000007A0
:104AD000FFFFFFFF80000003FFFFFFFF000000015A
:104AE000FFFFFFFE00000000FFFFFFFC00000000D2
:104AF0007FFFFFF800000000000000000000000041
:104B000000000000000000000000000000000000A5
:104B10000000000000000000000000000000000095
:104B20000000000000000000000000000000000085
:104B30007FFFFFF800000000FFFFFFFC0000000106
:104B4000FFFFFFFE00000003FFFFFFFF0000000764
:104B5000FFFFFFFF80000007FFFFFFFFC00000070F
:104B6000FFFFFFFF80000023FFFFFFFF0000007139
:104B7000FFFFFFFE000000F8FFFFFFFC000001FC4C
:104B80007FFFFFF8000003FE00000000000007FFA9
:104B900000000000000007FF00000000000007FF09
:104BA00000000000000007FF00000000000007FFF9
:104BB00000000000000007FF00000000000007FFE9
:104BC00000000000000007FF00000000000007FFD9
:104BD00000000000000007FF00000000000007FFC9
:104BE00000000000000007FF00000000000007FFB9
:104BF00000000000000007FF00000000000007FFA9
:104C000000000000000007FF00000000000007FF98
:104C100000000000000007FF00000000000007FF88
:104C200000000000000007FF00000000000007FF78
:104C300000000000000007FF00000000000007FF68
:104C400000000000000007FF00000000000007FF58
:104C500000000000000007FF00000000000007FF48
:104C600000000000000007FC00000000000007F04A
:104C70007FFFFFFC000007E1FFFFFFFE000007874A
:104C8000FFFFFFFF8000060FFFFFFFFFE000003F78
:104C9000FFFFFFFFF80000FFFFFFFFFFFE00007FA8
:104CA000FFFFFFFFFC00041FFFFFFFFFF0000707EF
:104CB000FFFFFFFFC0C007C1FFFFFFFF03C007F0FA
:104CC0007FFFFFFC0FC007FC000000003FC007FF94
:104CD00000000000FFC007FF00000001FFC007FF49
:104CE00000000001FFC007FF00000001FFC007FF38
:104CF00000000001FFC007FF00000001FFC007FF28
:104D000000000001FFC007FF00000001FFC007FF17
:104D100000000001FFC007FF00000001FFC007FF07
:104D200000000001FFC007FF00000001FFC007FFF7
:104D300000000001FFC007FF00000001FFC007FFE7
:104D400000000001FFC007FF00000001FFC007FFD7
:104D500000000001FFC007FF00000001FFC007FFC7
:104D600000000001FFC007FF00000001FFC007FFB7
:104D700000000001FFC007FF00000001FFC007FFA7
:104D800000000001FFC007FF00000001FFC007FF97
:104D900000000001FFC007FF00000001FFC007FF87
:104DA00000000001FFC007FF00000001FFC003FE7C
:104DB00000000000FF8001FC000000007F0000F800
:104DC0007FFFFFF83E000070FFFFFFFC1C0000218A
:104DD000FFFFFFFE08000003FFFFFFFF00000007CA
:104DE000FFFFFFFF80000007FFFFFFFFC00000077D
:104DF000FFFFFFFF80000003FFFFFFFF0000000137
:104E0000FFFFFFFE00000000FFFFFFFC00000000AE
:104E10007FFFFFF80000000000000000000000001D
:104E20000000000000000000000000000000000082
:104E30000000000000000000000000000000000072
:104E40000000000000000000000000000000000062
:104E50007FFFFFF800000000FFFFFFFC00000001E3
:104E6000FFFFFFFE00000003FFFFFFFF0000000741
:104E7000FFFFFFFF80000007FFFFFFFFC0000007EC
:104E8000FFFFFFFF88000003FFFFFFFF1C00000182
:104E9000FFFFFFFE3E000000FFFFFFFC7F00000061
:104EA0007FFFFFF8FF80000000000001FFC000004E
:104EB00000000001FFC0000000000001FFC0000072
:104EC00000000001FFC0000000000001FFC0000062
:104ED00000000001FFC0000000000001FFC0000052
:104EE00000000001FFC0000000000001FFC0000042
:104EF00000000001FFC0000000000001FFC0000032
:104F000000000001FFC0000000000001FFC0000021
:104F100000000001FFC0000000000001FFC0000011
:104F200000000001FFC0000000000001FFC0000001
:104F300000000001FFC0000000000001FFC00000F1
:104F400000000001FFC0000000000001FFC00000E1
:104F500000000001FFC0000000000001FFC00000D1
:104F600000000001FFC0000000000001FFC00000C1
:104F700000000001FFC0000000000001FFC00000B1
:104F8000000000007FC00000000000003FC00000E3
:104F9000000000000FC000000000000003C000007F
:104FA0000000000001C00000000000000040000000
:104FB00000000000000000000000000000000000F1
:104FC00000000000000000000000000000000000E1
:104FD0000000000000C000000000000003C000004E
:104FE000000000000FC00000000000003FC00000F3
:104FF00000000000FFC0000000000001FFC0000032
:1050000000000001FFC0000000000001FFC0000020
:1050100000000001FFC0000000000001FFC0000010
:1050200000000001FFC0000000000001FFC0000000
:1050300000000001FFC0000000000001FFC00000F0
:1050400000000001FFC0000000000001FFC00000E0
:1050500000000001FFC0000000000001FFC00000D0
:1050600000000001FFC0000000000001FFC00000C0
:1050700000000001FFC0000000000001FFC00000B0
:1050800000000001FFC0000000000001FFC00000A0
:1050900000000001FFC0000000000001FFC0000090
:1050A00000000001FFC0000000000001FFC0000080
:1050B00000000001FFC0000000000001FFC0000070
:1050C00000000001FFC0000000000001FFC0000060
:1050D00000000000FF800000000000007F000000D2
:1050E000000000003E000000000000001C00000066
:1050F00000000000080000000000000000000000A8
:10510000000000000000000000000000000000009F
:10511000000000000000000000000000000000008F
:10512000000000000000000000000000000000007F
:10513000000000000000000000000000000000006F
:10514000000000000000000000000000000000005F
:10515000000000000000000000000000000000004F
:10516000000000000000000000000000000000003F
:105170007FFFFFF800000000FFFFFFFC00000001C0
:10518000FFFFFFFE00000003FFFFFFFF000000071E
:10519000FFFFFFFF80000007FFFFFFFFC0000007C9
:1051A000FFFFFFFF88000023FFFFFFFF1C000071CF
:1051B000FFFFFFFE3E0000F8FFFFFFFC7F0001FC49
:1051C0007FFFFFF8FF8003FE00000001FFC007FF24
:1051D00000000001FFC007FF00000001FFC007FF43
:1051E00000000001FFC007FF00000001FFC007FF33
:1051F00000000001FFC007FF00000001FFC007FF23
:1052000000000001FFC007FF00000001FFC007FF12
:1052100000000001FFC007FF00000001FFC007FF02
:1052200000000001FFC007FF00000001FFC007FFF2
:1052300000000001FFC007FF00000001FFC007FFE2
:1052400000000001FFC007FF00000001FFC007FFD2
:1052500000000001FFC007FF00000001FFC007FFC2
:1052600000000001FFC007FF00000001FFC007FFB2
:1052700000000001FFC007FF00000001FFC007FFA2
:1052800000000001FFC007FF00000001FFC007FF92
:1052900000000001FFC007FF00000001FFC007FF82
:1052A000000000007FC007FC000000003FC007F0C6
:1052B0007FFFFFFC0FC007E1FFFFFFFE03C0078772
:1052C000FFFFFFFF81C0060FFFFFFFFFE040003F31
:1052D000FFFFFFFFF80000FFFFFFFFFFFE00007F62
:1052E000FFFFFFFFFC00041FFFFFFFFFF0000707A9
:1052F000FFFFFFFFC0C007C1FFFFFFFF03C007F0B4
:105300007FFFFFFC0FC007FC000000003FC007FF4D
:1053100000000000FFC007FF00000001FFC007FF02
:1053200000000001FFC007FF00000001FFC007FFF1
:1053300000000001FFC007FF00000001FFC007FFE1
:1053400000000001FFC007FF00000001FFC007FFD1
:1053500000000001FFC007FF00000001FFC007FFC1
:1053600000000001FFC007FF00000001FFC007FFB1
:1053700000000001FFC007FF00000001FFC007FFA1
:1053800000000001FFC007FF00000001FFC007FF91
:1053900000000001FFC007FF00000001FFC007FF81
:1053A00000000001FFC007FF00000001FFC007FF71
:1053B00000000001FFC007FF00000001FFC007FF61
:1053C00000000001FFC007FF00000001FFC007FF51
:1053D00000000001FFC007FF00000001FFC007FF41
:1053E00000000001FFC007FF00000001FFC003FE36
:1053F00000000000FF8001FC000000007F0000F8BA
:105400007FFFFFF83E000070FFFFFFFC1C00002143
:10541000FFFFFFFE08000003FFFFFFFF0000000783
:10542000FFFFFFFF80000007FFFFFFFFC000000736
:10543000FFFFFFFF80000003FFFFFFFF00000001F0
:10544000FFFFFFFE00000000FFFFFFFC0000000068
:105450007FFFFFF8000000000000000000000000D7
:10546000000000000000000000000000000000003C
:10547000000000000000000000000000000000002C
:10548000000000000000000000000000000000001C
:105490007FFFFFF800000000FFFFFFFC000000019D
:1054A000FFFFFFFE00000003FFFFFFFF00000007FB
:1054B000FFFFFFFF80000007FFFFFFFFC0000007A6
:1054C000FFFFFFFF88000023FFFFFFFF1C000071AC
:1054D000FFFFFFFE3E0000F8FFFFFFFC7F0001FC26
:1054E0007FFFFFF8FF8003FE00000001FFC007FF01
:1054F00000000001FFC007FF00000001FFC007FF20
:1055000000000001FFC007FF00000001FFC007FF0F
:1055100000000001FFC007FF00000001FFC007FFFF
:1055200000000001FFC007FF00000001FFC007FFEF
:1055300000000001FFC007FF00000001FFC007FFDF
:1055400000000001FFC007FF00000001FFC007FFCF
:1055500000000001FFC007FF00000001FFC007FFBF
:1055600000000001FFC007FF00000001FFC007FFAF
:1055700000000001FFC007FF00000001FFC007FF9F
:1055800000000001FFC007FF00000001FFC007FF8F
:1055900000000001FFC007FF00000001FFC007FF7F
:1055A00000000001FFC007FF00000001FFC007FF6F
:1055B00000000001FFC007FF00000001FFC007FF5F
:1055C000000000007FC007FC000000003FC007F0A3
:1055D0007FFFFFFC0FC007E1FFFFFFFE03C007874F
:1055E000FFFFFFFF81C0060FFFFFFFFFE040003F0E
:1055F000FFFFFFFFF80000FFFFFFFFFFFE00007F3F
:10560000FFFFFFFFFC00001FFFFFFFFFF000000790
:10561000FFFFFFFFC0C00001FFFFFFFF03C000004E
:105620007FFFFFFC0FC00000000000003FC0000033
:1056300000000000FFC0000000000001FFC00000EB
:1056400000000001FFC0000000000001FFC00000DA
:1056500000000001FFC0000000000001FFC00000CA
:1056600000000001FFC0000000000001FFC00000BA
:1056700000000001FFC0000000000001FFC00000AA
:1056800000000001FFC0000000000001FFC000009A
:1056900000000001FFC0000000000001FFC000008A
:1056A00000000001FFC0000000000001FFC000007A
:1056B00000000001FFC0000000000001FFC000006A
:1056C00000000001FFC0000000000001FFC000005A
:1056D00000000001FFC0000000000001FFC000004A
:1056E00000000001FFC0000000000001FFC000003A
:1056F00000000001FFC0000000000001FFC000002A
:1057000000000001FFC0000000000001FFC0000019
:1057100000000000FF800000000000007F0000008B
:105720007FFFFFF83E000000FFFFFFFC1C000001B0
:10573000FFFFFFFE08000003FFFFFFFF0000000760
:10574000FFFFFFFF80000007FFFFFFFFC000000713
:10575000FFFFFFFF80000003FFFFFFFF00000001CD
:10576000FFFFFFFE00000000FFFFFFFC0000000045
:105770007FFFFFF8000000000000000000000000B4
:105780000000000000000000000000000000000019
:105790000000000000000000000000000000000009
:1057A00000000000000000000000000000000000F9
:1057B00000000000000000000000000000000000E9
:1057C00000000000000000000000000000000000D9
:1057D00000000000000000000000000000000000C9
:1057E00000000000000000000000000000000000B9
:1057F00000000000000000000000000000000000A9
:105800000000000000000000000000000000000098
:105810000000000000000000000000000000000088
:105820000000000000000000000000000000000078
:105830000000000000000000000000000000000068
:105840000000000000000000000000000000000058
:105850000000000000000000000000000000000048
:105860000000000000000000000000000000000038
:105870000000000000000000000000000000000028
:105880000000000000000000000000000000000018
:105890000000000000000000000000000000000008
:1058A00000000000000000000000000000000000F8
:1058B00000000000000000000000000000000000E8
:1058C00000000000000000000000000000000000D8
:1058D00000000000000000000000000000000000C8
:1058E00000000000000000000000000000000000B8
:1058F0007FFFFFF800000000FFFFFFFC0000000139
:10590000FFFFFFFE00000003FFFFFFFF0000000796
:10591000FFFFFFFF80000007FFFFFFFFC000000741
:10592000FFFFFFFF80000003FFFFFFFF00000001FB
:10593000FFFFFFFE00000000FFFFFFFC0000000073
:105940007FFFFFF8000000000000000000000000E2
:105950000000000000000000000000000000000047
:105960000000000000000000000000000000000037
:105970000000000000000000000000000000000027
:105980000000000000000000000000000000000017
:105DD000F05D000800000020300000005C010008B9
:105DE000205E0008300000206006000078010008F6
:105DF00000A24A04000000000000000001020304A9
:105E00000607080902040608000000000102030456
:105E1000010203040607080900000000000000005A
:0400000508000121CD
:00000001FF
